:1000000025C43FC43EC43DC43CC43BC43AC491C6AD
:1000100038C437C436C435C434C406C62BC631C44C
:1000200030C42FC42EC42DC47AC6020408100102A5
:100030000201010201000002100408402002020136
:10004000010100000080805F8080808003000380C9
:1000500080147F147F14242A7F2A122313086462D9
:10006000364956205005038080801C224180804103
:10007000221C808022146B142208083E080850308D
:100080008080800808080880606080808060100898
:1000900004033E41413E80427F4080806251494698
:1000A0008022414936801814127F802745453980C7
:1000B0003C4A49318001710D03803649493680063A
:1000C00049291E803636808080563680808008140C
:1000D0002241801414141480412214088002510912
:1000E0000680324979413E7E09097E807F49493642
:1000F000803E414122807F41413E807F494941808D
:100100007F090901803E49493A807F08087F804184
:100110007F4180802040403F807F081463807F4083
:100120004040807F020C027F7F06187F803E414165
:100130003E807F090906803E41215E807F09196665
:1001400080264949328001017F01013F40403F80C4
:1001500007186018073F4038403F631408146303D2
:100160000478040361594543807F41418080030442
:1001700008106041417F8080020102808040404041
:100180004080030480808020545478807F48483029
:100190008038444428803844447F80385454488010
:1001A000047E05018048545438807F080870807AA6
:1001B0008080808020403A80807F08146280417F68
:1001C0004080807C047804787C040478803844443F
:1001D00038807C242418801824247C8078040480AF
:1001E000804854542480043F4444803C40407C80F8
:1001F0000C3040308C3C4030403C44281028444C6B
:1002000050503C8064544C448008364180807F804C
:100210008080804136088080080408100880808033
:1002200080801C2A4949221F047F4040201210125E
:1002300020102220221021545479807914147980BE
:10024000394444398039444439803D40407D803DC3
:1002500040403D807E25251A806C1A6F1A6C7D5AAD
:100260001E5A7D4E7B0F7B4E7C3A7E3A7C1C762E4E
:10027000761C1E347C341E0C1224120C081C3E7F8B
:10028000807F3E1C0880303F01627E303F028080CC
:100290001E3D777331607E7B7E60205F2380807E91
:1002A0007A7A7F80034579450310282428100814A2
:1002B0002A1408000000000036360836361E143CAA
:1002C000287844241D244442241D620108651C2210
:1002D0004146241D244C08443D44084C241D24461A
:1002E00001621D620142241D24427C4657467C7FE8
:1002F0002A2A7F802A7F417F2A0A0055000A304837
:100300004D33070629792906081C2A080808082AF7
:100310001C08EB0786075D074B07F006E006BC06E6
:10032000A7069C06F105910577051205E9049804D6
:100330001004AB03780359033A037F7F7F7F7F1C50
:100340001C1C1C1C080808080808080808080008E5
:100350000808000000080000FF1C3E773E1C3E77A6
:1003600063773E7763416377634108416341081CCB
:100370000841081C3E1C08FF4040414040404043AB
:10038000404040404540404040494040404051404E
:10039000404040214040404051404040484148405A
:1003A00048404140484040414040FF00027D00003D
:1003B00000017C020000007A0000000872040000C6
:1003C00008601000001068000000204010000000CD
:1003D00020000000000000000000000000000000FD
:1003E00000000000300000007C543800793D243DBE
:1003F000797B3F163F7B7E7C187C7E7C0810087CD6
:10040000700810087060082010601040002000FF85
:100410000C40013006300104401840061001600114
:100420001840020003600108010C404260065021A0
:100430002420582013581128100E680A101108683B
:100440000C1112086B081614096C0910100E680ABA
:1004500010130C680C1116086B081214096C0814A0
:10046000100A6808136F7717776F1009680A106F02
:100470007717776F110C680B101608690C111409A7
:100480006A1016100B7C102C2016601340412C4073
:100490000C400360002801FF403C433C40407C434B
:1004A0007C40403C433C40407C437C40403C433C9F
:1004B00040407C437C40205E215E20106F106F1016
:1004C0000877087708047B047B0402750275020133
:1004D000680168012050205020401020004020007A
:1004E0004000404000400000FF404040404040602D
:1004F0005048444464544C44446C546C44446C54DC
:100500006C7C446C556E7C446E556E7C7C6E556E76
:100510007CFF4040090100004541000003014040CC
:100520000005014040000941400000504101000029
:1005300060410100004051010000004151000000F5
:100540000041490000004141080000404501000011
:100550000541400003014040010500404000090101
:100560004040001001414000204141000040414115
:10057000000040410100FF2050502000304848302A
:100580000006090906000102020100000101000045
:10059000FF0300000000030000000007000000004F
:1005A000060200000005060000000C06000000081E
:1005B0000E0000000A0C040000080A0C00000418D9
:1005C0000C000008101C0000001418080000101493
:1005D00018000008301800001020380000002830F3
:1005E000100000202830000000000000002028300B
:1005F000FF000007000000000E00000008080800CF
:100600001010100000202020000040434300004054
:100610004646000040404C0C004040401818404006
:100620004060600000002020404040606000010702
:10063000444000020E48400018084C40301018405A
:1006400040602030404060273440407E30304040A1
:100650007E313340407E323640407E303644407EEC
:1006600030304C487E303050587E303060705E10F4
:100670001040507E303060707C202040607C21270C
:1006800044607C222E48607C38284C607C3B2B4C9C
:10069000607C3E2E4C607C3F2F4D60FF552A552AD2
:1006A000552A552A552AFF10101010100810100F47
:1006B0007010100808101010101010FF00262026CF
:1006C00000002620260000262026000026202400E8
:1006D000002620260000262026001026202610FFB7
:1006E00000001C0000003E223E007F4141417FFF90
:1006F00001000000000200010000040002000008E8
:100700000104000110020800022004110004410845
:10071000220008421044011045204802204A40505F
:1007200004415440600842684160114470426022B4
:100730004870446045507048604A50705060546042
:1007400070606068607060607060FF084428100826
:10075000040204085030100804040201FF010000E4
:1007600000000202010000060909060000304848A6
:100770003000205050200030484830000006090961
:100780000000000102FF785C6878717C38747C7A24
:1007900078506262787C606170687A6030787470DA
:1007A00079705269607C68706150667078206871F9
:1007B00060725074797062687270306174617850E0
:1007C000707A74314068441068703460284A605808
:1007D00060607038661860707842195864702970CB
:1007E000703A7854707051786A70FF142A49493E03
:1007F000001C2A493E003E493E087F2A1C08082268
:100800001C0808081C000808080008080808080850
:100810000808000808080000080800000008000098
:100820000000000000000C0000000C1200000C1280
:1008300024000C1224120C1224120CFF321E120B74
:10084000070503020001020305080D1511241FBE50
:10085000CFE5D1E0DEBFCDBF10E0A0E6B0E0EEE82E
:10086000FFE002C005900D92A836B107D9F711E05C
:10087000A8E6B0E001C01D92A933B107E1F704D3A7
:1008800084C3BECBCF93DF93CDB7DEB7C350CDBF0C
:1008900080913401853018F01092340103C08F5FCD
:1008A0008093340120913401E0913301F0E0E55967
:1008B000FF4FE20FF11D308119821A821B8280E006
:1008C00090E030FF11C0FC01EF5CFF4F4491FC0150
:1008D000E65DFF4FE491A1E0B0E0AC0FBD1FA40FB7
:1008E000B11D4C914E2B4C93369501968730910556
:1008F00041F780E090E0281789F0FC01E35CFF4FAE
:100900003491FC01E85CFF4FE491A1E0B0E0AC0F52
:10091000BD1FA30FB11D3C913E2B3C93019685302A
:10092000910549F78BB38C7F9981892B8BBB88B359
:1009300081789A81892B88BB82B3817E9B81892BA8
:1009400082BBCD5FCDBFDF91CF910895F09135018E
:100950008F2F8F704F2F50E0BA0160717070E0914F
:100960003301F4FF02C0E81B01C0E80FA09136017B
:100970008E2F90E004962A2F30E082179307F4F030
:1009800080913801882321F081508093380114C070
:10099000809137018093380145FF05C080E18F27A2
:1009A0008093350109C06115710521F0A550A09310
:1009B000330102C01092330181E00895E0933301C6
:1009C00080E008958F706370613019F040933801B2
:1009D00002C0109238016295682B609335014093F4
:1009E00037010895109233011092360110926B0076
:1009F00010926C0010926D0010926E0010926F00B9
:100A00000895F0DF1092350110923701089520917A
:100A100036010BC0FC0134913F3F49F00196E22FB3
:100A2000F0E0E559FF4F30832F5F283C98F3209387
:100A30003601089590913601983C40F4E92FF0E09A
:100A4000E559FF4F80839F5F9093360108958F3D56
:100A500049F0843C61F0863D79F08C3D79F0843E2C
:100A600079F002C08AE811C0863F61F002C085E8D3
:100A70000CC08C3F49F009C087E807C089E805C071
:100A800084E803C086E801C088E88052813910F507
:100A9000E82FF0E0CF01880F991F880F991FEE5BB8
:100AA000FF4FE80FF91F8091360195E001C0F90171
:100AB0009F012F5F3F4FE491E7FD0AC0883C30F46F
:100AC000A82FB0E0A559BF4FEC938F5F915079F7F5
:100AD00080933601089583E08ABB8EE787BB8EE161
:100AE00081BB8BB38C6F8BBB88B3816888BB82B3AF
:100AF000816E82BB10BE85E083BF84E086BF87E243
:100B00008CBF89B7856089BF87E689B912B880E94B
:100B10008AB986E083B90895CF9321D2C82F83FF85
:100B200002C085E001C081E06C2F661F6627661F4A
:100B3000660FEC2FE295E770F0E0EC5BF74F449125
:100B400041DFC770EC2FF0E0E45CF74FE491E093F5
:100B50006500CF910895EF92FF920F931F93CF936B
:100B6000DF930F92CDB7DEB77C01D6DF3BDF870185
:100B70000E5F1F4FC7010196F2D1982F42C0780136
:100B80009E37A1F40894E11CF11CC801E8D18E370E
:100B900061F1E82FE154E43140F5F0E0EE0FFF1F82
:100BA000EE5EFC4F8591949132DF1FC09F3F81F430
:100BB0000894E11CF11CC801D2D107C03BDF8701BA
:100BC0000F5F1F4FC701CBD178018F3FB9F70DC021
:100BD0009E3549F40894E11CF11CC801C0D1982F3E
:100BE0008E3509F0915C892F32DF87010F5F1F4F2F
:100BF000C701B5D1982F882321F080E099831ADFAF
:100C00009981992309F0BBCFC801A9D1882311F498
:100C100000E010E0C8010F90DF91CF911F910F917C
:100C2000FF90EF90089508951F920F920FB60F92C4
:100C300011242F933F934F935F936F937F938F93E1
:100C40009F93AF93BF93EF93FF9386B78C5F86BF5D
:100C500019DEFF91EF91BF91AF919F918F917F919D
:100C60006F915F914F913F912F910F900FBE0F9019
:100C70001F9018951F920F920FB60F9211242F9369
:100C80003F934F935F936F937F938F939F93AF9314
:100C9000BF93EF93FF938CB7895D8CBF8091660003
:100CA000882321F081508093660005C08091650003
:100CB000809366004BDE80B386FF08C0809164009D
:100CC00080FF1CC0809164008E7712C08091640008
:100CD00080FD05C081E08093640084E60DC08091B2
:100CE0006400813059F480916800882321F483E006
:100CF0008093640003C0815080936800FF91EF915E
:100D0000BF91AF919F918F917F916F915F914F9123
:100D10003F912F910F900FBE0F901F9018951F922B
:100D20000F920FB60F9211240F900FBE0F901F90CD
:100D300018951F920F920FB60F9211242F933F9385
:100D40004F935F936F937F938F939F93AF93BF93D3
:100D5000EF93FF936CB16B3119F486E080936900D7
:100D600080916900833009F441C0843028F48130D7
:100D700089F08230E0F409C0853081F0853008F4D4
:100D800042C0863009F06FC05FC0683409F06BC0A4
:100D900081E04FC06C3409F066C04AC06D3009F480
:100DA00062C06A3009F45FC082E0809369006E35EA
:100DB00011F483E03EC0643221F410926A0084E0B2
:100DC00038C080916000909161009C012F5F3F4F7F
:100DD00030936100209360006D3011F06A3021F48F
:100DE00060E0C5D085E025C0C2D03DC080916000E4
:100DF000909161009C012F5F3F4F309361002093E1
:100E00006000615C14C0962F9053913108F09750A8
:100E1000903190F080916000909161009C012F5F73
:100E20003F4F309361002093600060916A009FD033
:100E300082E08093690017C080916A008295807F6C
:100E4000890F80936A000FC080E090E09093630068
:100E5000809362009093610080936000C3DD81E81D
:100E6000F6DD10926900FF91EF91BF91AF919F91D4
:100E70008F917F916F915F914F913F912F910F9043
:100E80000FBE0F901F90189526DEBBDD789481E889
:100E9000DEDD8FEF94E3ACE081509040A040E1F7BD
:100EA00000C00000809162009091630054DE909336
:100EB000630080936200C0E1D0E4809164008823E5
:100EC00071F4809162009091630045DE909363001D
:100ED00080936200809164008068809364008091B8
:100EE0006400833051F77EDD82E8B1DD8FE79AE15F
:100EF000A6E081509040A040E1F700C0000072DD04
:100F00008FEF94E3ACE081509040A040E1F700C047
:100F10000000CABFD5B9CBBF85B7806585BF85B78F
:100F2000806285BF889585B78F7D85BF1BBE83E8AE
:100F30008EDD8FE79AE1A6E081509040A040E1F776
:100F400000C0000080E090E006DE90936300809394
:100F5000620080916400806880936400AECFE19964
:100F6000FECF1FBA8EBBE09A99278DB30895262F26
:100F7000E199FECF1CBA1FBA8EBB2DBB0FB6F894F9
:0E0F8000E29AE19A0FBE01960895F894FFCF11
:080F8E000000000080080100D2
:00000001FF
